:100000000C941E060C94CB260C94F8260C944606F1
:100010000C9446060C9446060C9446060C94460630
:100020000C9446060C9446060C9418120C94460642
:100030000C9446060C9446060C9446060C94460610
:100040000C9425270C9446060C94132B0C94562BD9
:100050000C9446060C9446060C9446060C944606F0
:100060000C9446060C9446067417D617B517B817A5
:10007000BB17BE17C117C417C717D617D017081953
:100080000A190A1908190A190A190A190A190A195A
:100090000A190A190A190A190A190A190A190A1948
:1000A0008E180A190A190A190A190A19FF170A19C2
:1000B0000A190A190A190A190A190A190A190A1928
:1000C0000A190A190A190A190A190A199A189A18FA
:1000D0009A189A189A189A189A189A189A180A191F
:1000E0000A190A190A190A190A19FF1799189918E9
:1000F000991899180A19A718AD18B318B918BF1884
:10010000C518CB18D118DB18E518EF18F9184018E6
:1001100002180A190A190A190A198E180A190A194D
:100120000A190A190A190A190A190A19981898189D
:10013000981898180A19A718AD18B318B918BF1845
:10014000C518CB18D118DB18E518EF18F9184018A6
:1001500002180A190A190A190A198E183D193D19A7
:100160003D193D193D193D193D193D193D193D19DF
:100170003D193D193D19541A541A541A541A541A57
:10018000541A82198C199619A019FE19081A171AEF
:10019000281AAF1BC41BD01BD91BE81B0D1C161C37
:1001A0005F1C281C561F5C1F621F691F771F991F49
:1001B000B71F456E746572206D656E752E2E2E000C
:1001C000546F67676C6564206D6963726F50504D42
:1001D00000546F67676C656420696E76657274653C
:1001E000642050504D2100546F67676C6564205443
:1001F00058206D7574696E672100546F67676C6570
:10020000642074656C656D65747279210050726F3D
:10021000746F636F6C206572726F72207769746897
:100220002052580054696D656F7574207768656E4B
:1002300020636F6E6E656374696E6720746F205201
:100240005800507265737320616E79206B65792058
:10025000746F2063616E63656C00436F6E6E6563DF
:1002600074696E6720746F2052582C20706F776508
:100270007220757020746865205258202877697440
:10028000682062696E6420706C7567206966206EF4
:100290006F74207573696E6720616C776179732064
:1002A00062696E642900546F67676C656420276912
:1002B0006D6D656469617465206F75747075742700
:1002C00000546F67676C65642027736C61766520E6
:1002D0006D6F64652700546F67676C6564202761E4
:1002E0006C776179732062696E642700546F676769
:1002F0006C65642050504D206368616E6E656C20A3
:100300006C696D69740053657420525353492069B8
:100310006E6A656374696F6E206368616E6E656C8A
:100320002028303D3D64697361626C652900536526
:10033000742050504D206D696E696D756D20737914
:100340006E630053657420626561636F6E20696E31
:1003500074657276616C0053657420626561636FC9
:100360006E2064656C617900536574206265616319
:100370006F6E206672657175656E637920696E2097
:10038000487A3A20303D64697361626C652C205074
:10039000783D504D52206368616E6E656C20782CFC
:1003A0002046783D465253206368616E6E656C202E
:1003B00078005365742050574D2073746F7020641B
:1003C000656C61792028302064697361626C6564B2
:1003D0002C20312D323535203D3D20302E317320FB
:1003E0002D2035306D696E29005365742050504DB5
:1003F0002073746F702064656C61792028302064EC
:10040000697361626C65642C20312D323535203D75
:100410003D20302E3173202D2035306D696E29003E
:10042000536574206661696C736166652064656CF0
:1004300061792028302064697361626C65642C20C6
:10044000312D323535203D3D20302E3173202D2089
:1004500035306D696E29002A2A2A2A2A2A2A2A2A50
:100460002A2A2A2A2A2A2A2A2A2A2A2A2A2A2A2AEC
:100470002A2A2A2A0052582041636B6564202D20C5
:1004800072657665727420737563636573736675E0
:100490006C21002A2A2A2A2A2A2A2A2A2A2A2A2AAD
:1004A0002A2A2A2A2A2A2A2A2A2A2A2A2A2A2A2AAC
:1004B000002A2A2A2A2A2A2A2A2A2A2A2A2A2A2AC6
:1004C0002A2A2A2A2A2A2A2A2A2A2A2A2A2A00528E
:1004D000582041636B6564202D20757064617465DC
:1004E000207375636365737366756C21002A2A2A0D
:1004F0002A2A2A2A2A2A2A2A2A2A2A2A2A2A2A2A5C
:100500002A2A2A2A2A2A2A2A2A2A0056616C696457
:100510002063686F69636573206172653A205B319F
:100520005D2D5B31365D20286368616E6E656C20E1
:10053000312D31362900536574206F7574707574D0
:1005400020666F7220706F727420005B585D2061AE
:10055000626F7274206368616E67657320616E6498
:10056000206578697420525820636F6E6669670051
:100570005B535D20736176652073657474696E6783
:100580007320746F205258005B525D20726576654F
:1005900072742052582073657474696E6773207486
:1005A0006F2064656661756C747300557365206EA9
:1005B000756D62657273205B312D445D20746F2010
:1005C0006564697420706F727473205B452D515D92
:1005D00020666F722073657474696E677300202DD6
:1005E00020726563656976657220636F6E66696700
:1005F000757261746F722C20727820737720000AF4
:100600000A6F70656E4C52536E67200053657420FC
:1006100073657269616C2062617564726174653AB8
:10062000200056616C69642063686F696365733A82
:100630002031202D20342B34202F2032202D203823
:10064000202F2033202D20382B34202F2034202D14
:10065000203132202F2035202D2031322B34202FF5
:100660002036202D20313600536574204368616E9A
:100670006E656C20636F6E6669673A20005365741F
:100680002044617461726174652028302D32293AEA
:10069000200053657420486F70206368616E6E653A
:1006A0006C7320286D61782032342C207365706162
:1006B000726174656420627920636F6D6D61732966
:1006C0002076616C69642076616C75657320312DCC
:1006D0003235353A2000536574206368616E6E656B
:1006E0006C2073706163696E6720287831306B48C5
:1006F0007A293A200053657420524620706F77653E
:10070000722028302D37293A200053657420524634
:10071000206D6167696320286865782920652E67E8
:100720002E20307844454144463030443A2000532E
:1007300065742062617365206672657175656E63AC
:10074000792028696E20487A293A20005B5A5D207A
:10075000656E746572207265636569766572206383
:100760006F6E66696775726174696F6E2075746902
:100770006C79005B465D20646973706C61792061FF
:10078000637475616C206672657175656E63696509
:10079000732075736564005B525D2063616C6375E3
:1007A0006C6174652072616E646F6D206B65792079
:1007B000616E6420686F70206C697374005B495DC2
:1007C000207265696E697469616C697A6520736508
:1007D0007474696E677320746F20736B65746368DB
:1007E0002064656661756C7473005B585D2072658A
:1007F00076657274206368616E67657320616E64EC
:100800002065786974206D656E75005B535D20739B
:100810006176652073657474696E677320746F20E8
:10082000454550524F4D20616E64206578697420B3
:100830006D656E7500557365206E756D62657273BA
:10084000205B302D395D20746F20656469742070E1
:100850006172616D657465727300202D2053797328
:1008600074656D20636F6E66696775726174696F18
:100870006E000A0A6F70656E4C52536E672000510D
:1008800029204F7574707574206265666F726520DB
:100890006C696E6B20283D465329203A2000502970
:1008A00020536C617665206D6F64652028657870D3
:1008B0006572696D656E74616C293A20004F29205C
:1008C00054696D65642042494E44206174207374FC
:1008D000617274757020203A20004E292050504DCE
:1008E000206F7574707574206C696D69746564200F
:1008F000202020203A200044495341424C454400E6
:100900004D292050504D205253534920746F20637D
:1009100068616E6E656C202020203A20004C2920F2
:1009200050504D206D696E696D756D2073796E63E1
:10093000202875732920203A200044495341424C15
:100940004544004B29204661696C736166652062ED
:100950006561636F6E20696E74762E2028312D32AA
:10096000353573293A20004A29204661696C736144
:10097000666520626561636F6E2064656C617920D5
:1009800028302D323535203D3E20313073202D204A
:100990003135306D696E293A200049292046616958
:1009A0006C7361666520626561636F6E206672714B
:1009B0002E203A200048292050574D2073746F7024
:1009C0002064656C6179202020202020203A2000BE
:1009D00047292050504D2073746F702064656C61FE
:1009E00079202020202020203A200046292046611E
:1009F000696C736166652064656C617920202020D4
:100A00002020203A200050574D206368616E6E65AB
:100A10006C200066756E6374696F6E3A2000292041
:100A2000706F72742000506F776572546F776572C3
:100A300000445446205548462033322D62697420C4
:100A400031306368004F70656E4C52536E67525878
:100A5000206D696E6920342F36636800466C7974A6
:100A6000726F6E2F4F72616E6765525820554846FF
:100A70002038636800525820747970653A20004429
:100A8000697361626C656400487A00203D3D200016
:100A900043616C63756C61746564207061636B6540
:100AA0007420696E74657276616C3A200042292068
:100AB0004D6963726F202868616C66292050504D23
:100AC000202020203A00412920496E766572746505
:100AD000642050504D20696E20202020203A0030A4
:100AE00029204D7574652062757A7A657220286DAB
:100AF0006F73746C79293A003929205365726961E2
:100B00006C2062617564726174653A00736D617224
:100B100074506F7274004672536B79005472616E38
:100B200073706172656E740044697361626C6564B0
:100B30000038292054656C656D657472793A2020FF
:100B40002020202020003729204368616E6E656CCC
:100B500020636F6E6669673A202000362920446161
:100B60007461726174652028302D32293A2020206A
:100B700000352920486F70206368616E6E656C7364
:100B80003A2020202020003429204368616E6E65C1
:100B90006C2073706163696E673A202000332920EE
:100BA000524620706F7765722028302D37293A2001
:100BB0002020003229205246206D616769633A2067
:100BC0002020202020202020003129204261736530
:100BD000206672657175656E63793A202020000089
:100BE00000000700020100000304060000000000EE
:100BF00000000001020408102040800102040810D7
:100C00002001020408102004040404040404040263
:100C10000202020202030303030303000000002395
:100C2000002600290000000000250028002B0000FD
:100C3000000000240027002A0000442C11241FBEBD
:100C4000CFEFD8E0DEBFCDBF13E0A0E0B1E0E6E932
:100C5000FEE502C005900D92AA39B107D9F716E05A
:100C6000AAE9B3E001C01D92AF35B107E1F71CE07E
:100C7000CCE3DCE004C02297FE010E944D2DCA3374
:100C8000D107C9F70E94802C0C94492F0C940000C6
:100C90008091A505813019F482E08093A5058091AB
:100CA000A505833019F484E08093A5050895A895DF
:100CB0000895DC01ED91FC910190F081E02D099502
:100CC000089561E083E10E94282860E083E10E94AA
:100CD000612882E08093B00085E08093B10061E0FC
:100CE00083E00E94282860E083E00E946128089544
:100CF000A4E0B0E0EEE7F6E00C94242D009749F173
:100D00009C0140E050E068E478EE81E090E00E94D1
:100D1000F52C61E083E129833A834B835C830E9455
:100D200061282981822F3A81932F4B81A42F5C81E6
:100D3000B52F8F3F9105A105B10529F020F08FEF68
:100D400090E0A0E0B0E08093B3008091B0008061BB
:100D500007C060E083E10E9461288091B0008F7E2F
:100D60008093B0002496E2E00C94402D60E08CE08B
:100D70000E94282861E08BE00E94282861E08DE035
:100D80000E94282860E082E00E94282861E084E038
:100D90000E942828089542E050E068E476E080E070
:100DA0000E94AB260895E3E0F0E089E080935700CD
:100DB000E491E67081E0E63009F080E00895CF9399
:100DC000DF93C82F0E94D306882381F0DFB781E02C
:100DD0008093A405F8940E94570688E180936000F0
:100DE000C0936000C1110E945706DFBFDF91CF9111
:100DF00008952091440530914505382748E0C90100
:100E0000880F991F37FF06C09C0151E2252750E14A
:100E1000352701C09C01415091F73093450520933F
:100E200044050895D82FC0E0CD1790F45E9A409AFB
:100E300064E670E080E090E00E949E275E98409813
:100E400064E670E080E090E00E949E27CF5FECCFE8
:100E50006CE271E080E090E00E949E27E4CF0F9367
:100E60001F93CF93DF93EC01062F15E0115051F043
:100E7000CE010E94302F081741F0602FCE010E9452
:100E8000382FF4CF82E00E941207DF91CF911F919B
:100E90000F910895A0E0B0E0E0E5F7E00C94162D86
:100EA000482E562EC0E0D0E0612C712CE12CF12CA4
:100EB00000E010E041100CC06090A30586E4689E3D
:100EC00030011124A9E1EA2EF12C0AE815E01EC038
:100ED00091E049120FC06090A305E6E46E9E3001D8
:100EE0001124FBE16F0E711CF9E2EF2EF12C06E4E8
:100EF00015E00CC082E0481209C078E1672E772423
:100F00007394EE24E394F12C03EA15E043018C0E74
:100F10009D1E10924505109244053401A62CA81878
:100F2000B12CC30101966C01AE14BF04A8F4A00E4D
:100F3000B11E511006C0C3010E94302FF5018083FD
:100F400005C0F5016081C3010E942F07F501808172
:100F50000E94F9063601E2CFC301511018C0C30147
:100F60000E94302FB82EC6010E94302F2B2D30E06A
:100F7000322F2227282B8091440590914505821716
:100F8000930779F4C0E0D0E05524539493CF360111
:100F9000609145050E942F0760914405C6010E949B
:100FA0002F07C05EDE4FC13E92E0D90708F482CF22
:100FB000852DCDB7DEB7E0E10C94322D87E3809329
:100FC000460580E092ECA1E0B0E080934705909365
:100FD0004805A0934905B0934A0587E080935305DF
:100FE00080EC92E9ADEEB9E180934B0590934C050E
:100FF000A0934D05B0934E0585E0809354058DEE8A
:101000009EEFADEABEED80934F0590935005A093FF
:101010005105B0935205E5E5F5E080E090E08630BB
:1010200028F4DC01AC59BC4F2C9101C020E0219385
:1010300001968831910599F782E080936D058AE0E9
:1010400080936E05089561E082E00E944A0708954A
:1010500060E082E00E944A078091A305843020F07E
:101060001092A3050E9423080895A1E0B0E0EBE3ED
:10107000F8E00C94242D89830E9428089091A30500
:101080008981981731F0843020F48093A3050E9461
:1010900023082196E2E00C94402D80EC91EDA8E924
:1010A000BBE180938B0590938C05A0938D05B09345
:1010B0008E0580E090E0A0E0B0E580938F059093EE
:1010C0009005A0939105B0939205E3E9F5E080E0E7
:1010D00081938F5F8031E1F70895A0E0B0E0E3E70E
:1010E000F8E00C941A2D0E947B276115710581058B
:1010F0009105C9F30E94B92D10924F051092500529
:101100001092510510925205C4E0C12CD12C7601E9
:10111000CA9480904F0590905005A0905105B090D2
:101120005205BA2CA92C982C88240E94B42DA70112
:1011300096010E94F52C680D791D8A1D9B1D6093F8
:101140004F05709350058093510590935205C150FF
:1011500001F705E515E0E801C12CD12CB2E38B2E97
:10116000912CA12CB12C80E1E82E87E2F82E888109
:10117000882309F446C0D39419F40E94DE0741C0C5
:101180000E94B42DA50194010E94F52C21E0260FA8
:10119000E5E5F5E08E2F801B8C1520F481918213FC
:1011A000F9CFE9CF40915405249FA00111244E9D11
:1011B000C0014F9D900D5E9D900D1124AA2797FDB3
:1011C000A095BA2F40914B0550914C0560914D056B
:1011D00070914E05840F951FA61FB71F40918B0578
:1011E00050918C0560918D0570918E0548175907B7
:1011F0006A077B0708F4BFCF2993C39488E1C8121C
:10120000B6CFCDB7DEB7ECE00C94362D61E080E0D0
:101210000E944A0761E081E00E944A07089560E069
:1012200080E00E944A07882331F060E081E00E945C
:101230004A07811108C00E944D080E94DE070E94E3
:101240006D080E94060908958436910520F4BC01BA
:1012500080E090E017C09C018E3B910528F42A5550
:101260003109AAE0B0E00CC0823D910528F4245B6E
:101270003109A4E6B0E004C02D5C3109A8E5B2E074
:101280000E948D2CA4E6B0E09B01AC010E949C2C36
:10129000089590E08C599F4F0E94240908958F92E1
:1012A0009F92AF92BF92CF92DF92EF92FF92CF9335
:1012B000FC01C0A5EC2FE770F0E0E45BFC4FA081DF
:1012C000B0E0C7FF03C024E130E002C02FE030E00F
:1012D000FC0197A183E1989FF0011124E25CFE4F8D
:1012E00080809180A280B380A20FB31F20E43FE1F1
:1012F0004DE750E00E94A72CA50194010E94D32C39
:101300008C2F887149F469017A01E0EDCE0EE7E097
:10131000DE1EE11CF11C1BC0C7FF05C060E47AE8BB
:101320008CE29EE004C060E07EEE8AEB9BE0690107
:101330007A01F8EBCF0EFBE0DF1EE11CF11CA501EA
:1013400094010E94D32CC20ED31EE41EF51EC701C9
:10135000B60169517C4F8F4F9F4F28EE33E040E03C
:1013600050E00E94D32CA8EEB3E00E949C2CCF91B9
:10137000FF90EF90DF90CF90BF90AF909F908F90B5
:1013800008958F3F910551F048F0811522E09207B2
:1013900038F08115934030F482E0089580E008959C
:1013A00081E0089583E00895A0E0B0E0EAEDF9E07F
:1013B0000C941F2DEB018A01B82FB695A0E028816F
:1013C0003981F80120832A813B8121832C813D8151
:1013D00022832E813F812383688179814A815B81C9
:1013E0002C813D81EE81FF819F2F9295990F990F5E
:1013F000907C272F2370922B252F2370220F220FF2
:10140000922B232F23702295207F922BF801948317
:101410000B5F1F4F2896AF5FBA1788F680FF24C076
:10142000888199810E94C109D82E8A819B810E945E
:10143000C109E82E8C819D810E94C109F82E8E8100
:101440009F810E94C109F0E4DF9EA001112490E178
:10145000E99E90011124242B282BE4E0FE9EB0018C
:101460001124262BF8012083CDB7DEB7E7E00C94DA
:101470003B2D803223E0920708F1883E23E092075B
:1014800040F48F519340E4E096958795EA95E1F713
:101490000895803D27E0920718F48C5D93400895ED
:1014A000883928E0920768F4885C974074E0969544
:1014B00087957A95E1F78D509C4F089580E090E0F4
:1014C00008958FEF93E008958C30910540F4A4E0E7
:1014D000880F991FAA95E1F7885D9C4F0895843F76
:1014E00023E0920718F484529C4F0895811524E05C
:1014F000920740F48657934FF4E0880F991FFA95AE
:10150000E1F7089580E998E008959C0136952795C4
:1015100025753575821B930B9C0123733373969548
:1015200087959695879583739373820F931F9C017C
:1015300054E0369527955A95E1F7280F391F2F70FB
:101540003F7041E051E0249FC001259F900D349FE2
:10155000900D1124892F08952D98882319F00000EB
:101560002B9A02C000002B9800002D9A00000895CD
:101570002D9A000083B12D98000082958170089506
:10158000CF93DF93D82F5C9A2D985C98C8E08D2F6D
:1015900080780E94AC0ADD0FC150C9F72D98DF9109
:1015A000CF9108958F770E94C00A0895CF93DF935B
:1015B000D82FC8E08D2F80780E94AC0ADD0FC15073
:1015C000C9F72D98DF91CF910895CF93DF932D9890
:1015D000C8E080E0D82FDD0F0E94B80A8D0FC150FF
:1015E000C9F7DF91CF9108950E94D20A0E94E50ABF
:1015F0005C9A0895A1E0B0E0E0E0FBE00C94242DBB
:10160000806869830E94C00A6981862F0E94D60A79
:101610005C9A2196E2E00C94402DCF93C0914F0547
:10162000C827E82FF0E0EA5BFA4F678589E70E9458
:10163000FA0A6C2F8DE30E94FA0A6C2F82E40E9452
:10164000FA0ACF91089586E20E94F40A0895CF9392
:10165000DF93EC016C818CE10E94FA0A6D818DE1CF
:101660000E94FA0A6E818EE10E94FA0A6F8180E27E
:101670000E94FA0A688581E20E94FA0A698582E27C
:101680000E94FA0A6A8583E20E94FA0A6B8584E264
:101690000E94FA0A6C8585E20E94FA0A6D858AE248
:1016A0000E94FA0A6E858EE60E94FA0A6F858FE61E
:1016B0000E94FA0A688980E70E94FA0A698981E72C
:1016C0000E94FA0A6A8982E70E94FA0ADF91CF91A2
:1016D0000895CF92DF92EF92FF92CF93DF936B0149
:1016E0007C01C11488E3D8068CE9E8068CE1F80691
:1016F00028F5C701B60120E836E948E950E00E9424
:10170000D32CE901689760E879E687E69FEF0E94AD
:10171000AF2C6C0D7D1D8E1D9F1DF2E0660F771F97
:10172000881F991FFA95D1F721E732E040E050E099
:101730000E94D32CF22EE32E80E421C0C701B60113
:1017400020E03DE241E351E00E94D32CE90168979B
:1017500060E073ED8EEC9EEF0E94AF2C6C0D7D1D52
:101760008E1D9F1D660F771F881F991F21E732E08E
:1017700040E050E00E94D32CF22EE32E80E66C2F46
:101780006F71680F85E70E94FA0A6E2D86E70E9446
:10179000FA0A6F2D87E70E94FA0ADF91CF91FF9036
:1017A000EF90DF90CF900895682F8DE60E94FA0A9F
:1017B00008958F929F92AF92BF92CF92DF92EF9255
:1017C000FF92CF93DF93D82F83E00E94F40A809397
:1017D000430584E00E94F40A8093420560E086E0BD
:1017E0000E94FA0A61E087E00E94FA0A6FE789E046
:1017F0000E94FA0A65E08AE00E94FA0A62E18BE040
:101800000E94FA0A65E18CE00E94FA0A6DEF8DE011
:101810000E94FA0A60E08EE00E94FA0ADD2319F0C5
:101820008BE291E008C020916D0533E1239FC00158
:101830001124825C9E4F0E94270B6CE880E30E947B
:10184000FA0A6FE082E30E94FA0A62E483E30E94EC
:10185000FA0A80916E0587FF02C064E101C06AE068
:1018600084E30E94FA0A6AE285E30E94FA0A6DE2C2
:1018700086E30E94FA0A64ED87E30E94FA0A60E0B8
:1018800088E30E94FA0A60E089E30E94FA0AD11113
:1018900009C0C0904F05D0905005E0905105F090E0
:1018A000520507C0C5E8CC2EC1ECDC2EED2CCEEDE8
:1018B000FC2ECAE38F2C9924AA24BB24682D8C2FDC
:1018C0000E94FA0A682D85E08C0F0E94FA0AFE2C0D
:1018D000ED2CDC2CCC24CF5FCE3361F76FEF83E4AB
:1018E0000E94FA0A6FEF84E40E94FA0A6FEF85E41F
:1018F0000E94FA0A6FEF86E40E94FA0ADD2311F0D3
:1019000066E002C0609153058DE60E94FA0A60E02D
:1019100089E70E94FA0A609154058AE70E94FA0A50
:1019200060E083E70E94FA0A60E084E70E94FA0A16
:10193000D11109C060914B0570914C0580914D0506
:1019400090914E0504C060EC72E98DEE99E10E9421
:10195000690BDF91CF91FF90EF90DF90CF90BF9018
:10196000AF909F908F90089561E087E00E94FA0AFF
:1019700064E28EE70E94FA0A63E088E00E94FA0AB5
:1019800060E088E00E94FA0A65E087E00E94FA0AB7
:1019900062E085E00E94FA0A83E00E94F40A8093E4
:1019A000430584E00E94F40A80934205089583E091
:1019B0000E94F40A8093430584E00E94F40A809315
:1019C000420561E087E00E94FA0A6AE070E080E088
:1019D00090E00E949E270E94B40C00000895CF92D0
:1019E000DF92FF920F931F93CF93DF931F92CDB798
:1019F000DEB7082F162F8EE399830E94FA0AF02E85
:101A0000C02E9981D92E8C2D8F19811738F4F601AB
:101A100061916F018FE70E94FA0AF5CF64E085E0DB
:101A20000E94FA0A83E00E94F40A8093430584E04E
:101A30000E94F40A809342050E947B2760933E0532
:101A400070933F05809340059093410569E087E0DE
:101A50000E94FA0A81E08093A5050F90DF91CF9153
:101A60001F910F91FF90DF90CF9008950F931F93D8
:101A70000E94EF0C8091A505813099F40E947B278C
:101A800000913E0510913F052091400530914105A0
:101A9000601B710B820B930B603A76488140910575
:101AA00048F38091A505813031F46EE971E083EB54
:101AB00095E00E9467291F910F9108950F931F933E
:101AC0008091A505823021F41092A50581E020C007
:101AD0008091A5058130D9F40E947B2700913E05B5
:101AE00010913F052091400530914105601B710B1D
:101AF000820B930B613A76488140910540F061E09A
:101B000087E00E94FA0A1092A50582E001C080E0F9
:101B10001F910F910895CF93DF93EC014AE050E0BD
:101B20006D2F70E083EB95E00E94352A6EE283EB27
:101B300095E00E943929BE0184E0769567958A95E3
:101B4000E1F76F7077274AE050E083EB95E00E9461
:101B5000352A6EE283EB95E00E943929BE016F7051
:101B600077274AE050E083EB95E00E94352ADF9129
:101B7000CF910895882319F06AEA71E002C06EEAF5
:101B800071E083EB95E00E9467290895FF920F931F
:101B90001F93CF93DF9369EC7BE083EB95E00E948A
:101BA000132940914B0550914C0560914D05709162
:101BB0004E052AE030E083EB95E00E943C2A63EB7F
:101BC0007BE083EB95E00E94132940914F055091F3
:101BD0005005609151057091520520E130E083EB92
:101BE00095E00E943C2A6DE97BE083EB95E00E9442
:101BF00013294AE050E06091530583EB95E00E9481
:101C0000642A67E87BE083EB95E00E9413294AE0B1
:101C100050E06091540583EB95E00E94642A61E7EF
:101C20007BE083EB95E00E941329C5E5D5E0F12C1C
:101C30008E0188818823A9F0FF2031F061EB71E0EB
:101C400083EB95E00E94362921964AE050E0F801A6
:101C5000608183EB95E00E942D2AF394F8E1FF1256
:101C6000E7CF83EB95E00E9441296BE57BE083EBB6
:101C700095E00E9413294AE050E060916D0583EBE6
:101C800095E00E94642A66E47BE083EB95E00E9485
:101C90001329E0916E05E770F0E0EE0FFF1FEC5A9C
:101CA000FC4F6081718183EB95E00E94672961E3BD
:101CB0007BE083EB95E00E94132980916E0588718B
:101CC000883069F028F4811113C068E27BE00CC011
:101CD000803141F0883161F46CE07BE005C06CE15B
:101CE0007BE002C066E17BE083EB95E00E94552932
:101CF00068EF7AE083EB95E00E9413294091470555
:101D0000509148056091490570914A052AE030E0FC
:101D100083EB95E00E943C2A6FED7AE083EB95E03F
:101D20000E94132980918F0580710E94BA0D66EC84
:101D30007AE083EB95E00E94132980918F058074EF
:101D40000E94BA0D6DEA7AE083EB95E00E941329B8
:101D500080918F0580720E94BA0D60E97AE083EB72
:101D600095E00E94132986E495E00E944F09AB019B
:101D7000BC012AE030E083EB95E00E941E2A6BE86C
:101D80007AE083EB95E00E94132986E495E00E94B7
:101D90004F099B01AC0160E472E48FE090E00E9487
:101DA000D32CBA01A9012AE030E083EB95E00E9430
:101DB0001E2A68E87AE083EB95E00E945529CDB7AA
:101DC000DEB7E5E00C943D2D8F929F92AF92BF92CB
:101DD000CF92DF92EF92FF92811107C06FE77AE016
:101DE00083EB95E00E9455292FC090E00E942409C2
:101DF00024E630E040E050E00E94D32CCA01B90153
:101E00002AE030E040E050E00E94D32C49015A0122
:101E10006B017C012AE030E0B501A40183EB95E081
:101E20000E941E2A6EE283EB95E00E9439292AE087
:101E300030E0B701A60183EB95E00E941E2A63E71C
:101E400083EB95E00E947929FF90EF90DF90CF908F
:101E5000BF90AF909F908F9008951F93CF93DF9383
:101E600065E77AE083EB95E00E94132980916F0586
:101E7000813041F46CE57AE083EB95E00E945529CE
:101E800010E050C0823019F465E47AE0F5CF843078
:101E900019F461E37AE0F0CF853091F766E27AE0F9
:101EA000EBCFC12FD0E0C930D1050CF441C068E3BD
:101EB000610F83EB95E00E9439296EE17AE083EBB4
:101EC00095E00E941329BE016F5F7F4F4AE050E00A
:101ED00083EB95E00E94FD2963E17AE083EB95E0D6
:101EE0000E941329C159DA4FE981E03218F566E002
:101EF0007AE083EB95E00E9413298981803130F0EC
:101F00006FE373E083EB95E00E94362969816F707F
:101F100070E06F5F7F4F4AE050E083EB95E00E94F6
:101F2000062A1F5F80911A05181708F4BACF0FC050
:101F300061E3BECFEF70F0E0EE0FFF1FE659FC4FFC
:101F40006081718183EB95E00E946729EACF6BEE97
:101F500079E083EB95E00E941329809187050E9428
:101F6000E40E60ED79E083EB95E00E941329809107
:101F700088050E94E40E65EB79E083EB95E00E9412
:101F80001329809189050E94E40E6AE979E083EBC8
:101F900095E00E94132940917F0550918005609142
:101FA000810570918205411551056105710539F171
:101FB0002AE030E083EB95E00E943C2A67E679E076
:101FC00083EB95E00E941329809183050E944909C3
:101FD000AB01BC012AE030E083EB95E00E943C2A93
:101FE00063E479E083EB95E00E9413294AE050E036
:101FF0006091840583EB95E00E94642A06C06AE341
:1020000079E083EB95E00E9455296DE179E083EB5F
:1020100095E00E94132960918505709186054AE03C
:1020200050E083EB95E00E944E2A60E079E083EB7C
:1020300095E00E94132960917E05603450F470E0B1
:102040006F5F7F4F4AE050E083EB95E00E94062AE5
:1020500006C067EF78E083EB95E00E9455296AEDB2
:1020600078E083EB95E00E94132980917D0580FF45
:1020700003C063EB71E002C067EB71E083EB95E0B6
:102080000E9467296DEB78E083EB95E00E941329AD
:1020900080917D0582700E94BA0D6EE978E083EB35
:1020A00095E00E94132980917D0584700E94BA0DED
:1020B0006FE778E083EB95E00E94132980917D051E
:1020C00088700E94BA0DDF91CF911F9108950F93F0
:1020D0001F93CF93DF93209117052F3FA9F56FEF43
:1020E00075E083EB95E00E94132984E793E00E945A
:1020F0008B0D6EED75E083EB95E00E9413298091C6
:102100001805909119050E948B0D6BEA75E083EB21
:1021100095E00E94552968E875E083EB95E00E9400
:10212000552960E775E083EB95E00E9455296BE443
:1021300075E083EB95E00E94552983EB95E00E94C2
:1021400041290E942D0F68C012160CF065C033277C
:1021500027FD309580911A0590E0821793070CF4C3
:102160005BC066E375E083EB95E00E941329609104
:102170001705772767FD70954AE050E083EB95E0FF
:102180000E94062A6BE075E083EB95E00E9413291C
:1021900010E008E280911B051817D0F5C12FD0E0A0
:1021A000CC0FDD1FC45EDA4F288130E08091170527
:1021B000992787FD909501972817390739F56BEB1B
:1021C00071E083EB95E00E9436294AE050E0602FF1
:1021D00083EB95E00E942D2A6FEB71E083EB95E095
:1021E0000E943629E981EF70F0E0EE0FFF1FE659FB
:1021F000FC4F6081718183EB95E00E94362963EC8E
:1022000071E083EB95E00E9436290F5F1F5FC2CF1C
:1022100083EB95E00E944129DF91CF911F910F91AF
:102220000895FF920F931F93CF93DF93C5E5D5E0F9
:10223000F12C8E0188818823D1F165EC71E083EB6C
:1022400095E00E9436294AE050E06F2D83EB95E03F
:102250000E942D2A62ED71E083EB95E00E94362901
:102260002196F801208130E0A0E1B7E20E948D2C98
:102270009B01AC01A0915405B0E00E949C2CAB01E5
:10228000BC0180914B0590914C05A0914D05B091FA
:102290004E05480F591F6A1F7B1F2AE030E083EB71
:1022A00095E00E943C2AF394F8E1FF12C2CFCDB72B
:1022B000DEB7E5E00C943D2D1092B10485E6E2EB2B
:1022C000F4E0DF011D928A95E9F70895CF93C82FB6
:1022D0008F3719F0883009F045C0E091B104EE2342
:1022E000D9F1E150E093B104F0E0EE54FB4F1082DD
:1022F0006DE070E083EB95E00E945906C0E08091AC
:10230000B104C81760F4EC2FF0E0EE54FB4F60818D
:1023100070E083EB95E00E945906CF5FF0CF60E25A
:1023200070E083EB95E00E9459066DE070E083EB6E
:1023300095E00E945906C0E08091B104C81778F575
:10234000EC2FF0E0EE54FB4F608170E083EB95E002
:102350000E945906CF5FF0CF67E083EB95E00E94C3
:1023600039291DC08B3119F40E945C111AC08D30BF
:10237000C1F08A30B1F08091B104843668F76C2FD7
:1023800070E083EB95E00E945906E091B10481E092
:102390008E0F8093B104F0E0EE54FB4FC08380E0D9
:1023A00001C081E0CF910895CF93C82F0E947B2771
:1023B00060939A0470939B0480939C0490939D0473
:1023C000C093AF04CC2329F040E051EE60E070E010
:1023D00004C040E855E260E070E083EB95E00E94C5
:1023E000C32BCF91089590919E04492F4F7050E0D8
:1023F000BA016F5F7F4F292F30E0E4E035952795D4
:10240000EA95E1F76217730759F0FA01E156FB4FBD
:10241000808381E0890F8F70907F892B80939E0449
:1024200008956EE770E083EB95E00E9459060895E9
:102430001F920F920FB60F9211241F932F933F9369
:102440004F935F936F937F938F939F93AF93BF93BC
:10245000CF93DF93EF93FF93C0918600D0918700D5
:102460008091590490915A0420917B04211155C008
:102470009E01281B390B80918F0590919005A091AA
:102480009105B091920585FD02C036952795253CB2
:1024900049E03407B8F140910A0150E060E070E093
:1024A0001CE1B695A795979587951A95D1F7009752
:1024B000A105B10521F481E090E0A0E0B0E084172F
:1024C0009507A607B707D8F480910A018F3FB9F0A6
:1024D00040E080910A01481780F4842F90E0880F33
:1024E000991FFC01E55AFB4F20813181FC01E55F1A
:1024F000FE4F318320834F5FECCF10927C0410920B
:102500000A010BC02D3B82E0380720F080910A01C0
:102510008031D8F08FEF80930A01D0935A04C09392
:102520005904FF91EF91DF91CF91BF91AF919F91AE
:102530008F917F916F915F914F913F912F911F915B
:102540000F900FBE0F901F90189510910A0181E017
:10255000810F80930A01C9010E94390AE12FF0E03E
:10256000EE0FFF1FE55AFB4F91838083D6CF83E0A8
:10257000809380008AE98093810080918F0586FD99
:1025800005C0809181008064809381008FEF9FEF70
:10259000909389008093880080916F00806280937F
:1025A0006F0008956F3018F086958058089589E07F
:1025B000689F802D11240895A0E0B0E0E2EEF2E1E2
:1025C0000C941E2DC82F0E947B2700910A041091A5
:1025D0000B0420910C0430910D046B017C01C01A96
:1025E000D10AE20AF30A9701860149E8C41643E1D9
:1025F000D406E104F10410F010920E0460930A0472
:1026000070930B0480930C0490930D0420917B0431
:102610008FEF820F8230D8F5E0910E04EE2309F49B
:102620004EC1E13011F482E0B8C1E03108F034C1AC
:1026300081E08E0F80930E04F0E0E55AFB4FC083DB
:10264000803109F0ACC1EDE5F4E0213029F4A1813D
:10265000A695A695808108C080819181A92FA69515
:10266000A695A69596958795A03148F4B0E090E0A0
:10267000AA0FBB1FA55FBE4F11969C938E9310921D
:102680007C04329684E0EB36F807F9F688C12330F3
:1026900009F005C1E0910E04E11104C0CF3009F04A
:1026A0007EC10DC1E83148F481E08E0F80930E04A5
:1026B000F0E0E65AFB4FC08372C1E83109F0ECC08C
:1026C000C111EAC040E050E0ABE0CA01B3E0880FBE
:1026D000991FBA95E1F7A49F9001A59F300D112491
:1026E000F901E55AFB4F6081E1817E2F7770759586
:1026F0006795FC01EE0FFF1FE55FFE4F718360835E
:10270000F901E45AFB4FB081B695B695B695E181D3
:10271000FE2FF295FF0FF07E6F2F6B2BE695E6955F
:10272000E6957E2F777075956795FC01EE0FFF1F7C
:10273000E35FFE4F71836083F901E35AFB4FB08181
:10274000B295B695B695B370C181DC2FDD0FDD0F64
:102750006D2F6B2BC295C695C695C370E281E17053
:10276000EE0FEE0F7E2F7C2B75956795FC01EE0F1B
:10277000FF1FE15FFE4F71836083F901E15AFB4F58
:10278000B081B695E181FE2FF795FF27F7956F2F62
:102790006B2BE6957E2F777075956795FC01EE0F94
:1027A000FF1FEF5EFE4F71836083F901E05AFB4F1C
:1027B000B081B295BF70E181FE2FF295F07F6F2F4F
:1027C0006B2BE295EF707E2F777075956795FC0106
:1027D000EE0FFF1FED5EFE4F71836083F901EF592D
:1027E000FB4FB081BB1FBB27BB1FC181DC2FDD0F9F
:1027F0006D2F6B2BCC1FCC27CC1FE281E370EE0F2B
:102800007E2F7C2B75956795FC01EE0FFF1FEB5E0D
:10281000FE4F71836083F901ED59FB4FB081B6958E
:10282000B695E181FE2FF295FF0FFF0FF07C6F2F21
:102830006B2BE695E6957E2F777075956795FC0175
:10284000EE0FFF1FE95EFE4F71836083F901EC59C3
:10285000FB4F20812295269527703181E32FEE0FC3
:10286000EE0FEE0F6E2F622B732F729576957770A9
:1028700075956795FC01EE0FFF1FE75EFE4F7183B4
:1028800060834F5F5F4F4230510509F01ECF80914A
:10289000710483FF10927C0410920E0480C02430D7
:1028A00009F07DC060910E0461110BC0C83AB1F40B
:1028B000109245051092440588EA0E94F90681E0CD
:1028C0006CC0613019F4C093090404C0623031F463
:1028D000C09308048C2F0E94F9065AC0E0910804A6
:1028E0002E2F30E0220F331F462F50E0C9010296F1
:1028F000841795073CF0633268F7FA01E85AFB4FFA
:10290000C083E8CF2D5F3F4F8C2F90E0609144054E
:10291000709145054217530749F4982F8827862759
:102920009727909345058093440532C0681779072F
:1029300069F580910904813049F5E13118F080E1B1
:1029400080930804F0900804CCE5D4E000E010E0A7
:102950000F15D0F4FE013197808190E0982F8827E1
:102960002881822B63E0969587956A95E1F70E940E
:10297000390AF801EE0FFF1FE55FFE4F9183808358
:102980000F5F1F4F2296E4CF10927C0410920E042A
:1029900080910E04882319F08F5F80930E04CDB7C9
:1029A000DEB7E8E00C943A2DE82FF0E0E657FA4F56
:1029B000E185E03158F4F894F0E0EE0FFF1FE55F99
:1029C000FE4F208131817894C9010895E03121F0D2
:1029D000E13131F483E101C082E10E94BD28089514
:1029E00080E092E00895A2E2B0E0E9EFF4E10C9417
:1029F000142D9E012F5F3F4F80E1D9011D928A95D2
:102A0000E9F766ED71E083EB95E029A33AA30E9414
:102A100067290E94D70C1D8A1E8A1F8A188E312CA6
:102A2000212C00E0812C912C540170E4472E71EE92
:102A3000572E7DE9672E78E1772EE0E5CE2EE3EC88
:102A4000DE2EE12CF12C84EF91E0A0E0B0E08D8F40
:102A50009E8FAF8FB8A380EC91EDA8E9BBE1898F81
:102A60009A8FAB8FBC8F80E491EEADE9B8E1898B92
:102A70009A8BAB8BBC8B83EB95E00E947B2A892BD6
:102A800009F4E1C083EB95E00E94A82A9C0133275A
:102A90002C32310509F442C0ACF42332310509F07F
:102AA000ABC019821A821B821C821D821E821F8269
:102AB000188619861A861B861C861D861E861F860A
:102AC000188A60C02434310529F02335310509F412
:102AD000B2C092C064E483EB95E00E9439292AE0F9
:102AE00030E040E451EE6DE978E183EB95E00E943F
:102AF000C7296CE283EB95E00E9439292AE030E097
:102B000040EC51ED68E97BE183EB95E00E94C72939
:102B10006CE283EB95E00E947929ADCF0F5F043022
:102B200009F0A9CF29813A814B815C81A8EEB3E0FD
:102B30000E949C2C698B7A8B8B8B9C8B2D813E8188
:102B40004F8158850E949C2C698F7A8F8B8F9C8F28
:102B500029853A854B855C852D8F3E8F4F8F58A3F5
:102B60002D853E854F8558890E949C2C6B017C01E8
:102B700060323EE473078105910530F462E38CE135
:102B80000E94FA0A00E077CF603345E774078105B9
:102B9000910510F462E2F3CF60345CE975078105BA
:102BA000910510F466E2EBCF80E5C81683ECD806F9
:102BB000E104F10410F462E1E2CF90E6C9169AEE66
:102BC000D906E104F10410F465E1D9CFA0E7CA16F3
:102BD000A1E1DA06A1E0EA06F10410F461E0CFCF4A
:102BE000B0EACB16B6E8DB06B1E0EB06F10410F470
:102BF00063E0C5CF65E0C3CF10ED180F1A3008F0C1
:102C00003ACFE1E0F0E0EC0FFD1F24E0029FE00D81
:102C1000F11D11242081318142815381AAE0B0E06D
:102C20000E949C2C610F711D811D911D6083718319
:102C30008283938320CF49885A886B887C88812C33
:102C4000912C540118CF81149104A104B10489F48A
:102C5000C301B2010E94690B61E070E080E090E086
:102C60000E949E271D8A1E8A1F8A188E312C2224BC
:102C70002A948D8D9E8DAF8DB8A188169906AA06CF
:102C8000BB06D0F40E94230B2D893E894F89588DB5
:102C9000280F311D411D511D2D8B3E8B4F8B588FA1
:102CA000381608F4382E821508F4282E3FEF831AC0
:102CB000930AA30AB30A56C0C301B20128EE33E057
:102CC00040E050E00E94D32CBA01A9012AE030E094
:102CD00083EB95E00E941E2A6CE283EB95E00E9454
:102CE00039294AE050E0632D83EB95E00E942D2ABC
:102CF0006CE283EB95E00E9439296D897E898F898A
:102D0000988DA50194010E94D32CBA01A9012AE053
:102D100030E083EB95E00E941E2A6CE283EB95E0A5
:102D20000E9439294AE050E0622D83EB95E00E9431
:102D30002D2A6CE283EB95E00E9479294C0C5D1CF6
:102D40006E1C7F1C898D9A8DAB8DBC8D841595056D
:102D5000A605B70520F449885A886B887C88812CA1
:102D6000912C540129893A894B895C89283E33404A
:102D70004105510509F07FCEA296E2E10C94302D79
:102D8000ACE1B0E0E6ECF6E10C941E2D0E947B274E
:102D90006B017C0181E00E94D90B14E703E01983E9
:102DA00061E0CE0101960E94360D0093A5050E94B8
:102DB000B40C6AEF70E080E090E00E949E27809162
:102DC000A505833089F483EB95E00E947B2A892B4B
:102DD00059F40E947B276C197D098E099F09603880
:102DE000734C894C9140D8F28091A505833009F449
:102DF0004FC08FE70E94D20A0E94E50A898384357A
:102E000011F083E05CC00E94E50A109218058093DF
:102E100019050E94E50A2091180530911905280F1F
:102E2000311D30931905209318050E94E50A8093FF
:102E30001A050E94E50A80931B05813110F7F12CD9
:102E40000F2D10E080911B0590E0880F991F081747
:102E5000190740F40E94E50AF801E45EFA4F808306
:102E6000F394EECF80E7898361E0CE0101960E9462
:102E7000360D83E08093A5050E94B40C62E370E0F8
:102E800080E090E00E949E278091A505833011F498
:102E900082E015C08FE70E94D20A0E94E50A89836A
:102EA000803509F0AECF0FE615E00E94E50AF80183
:102EB00081938F01F5E00A381F07B9F781E06C961E
:102EC000E8E00C943A2D80911705992787FD90959D
:102ED000A92FB92FFC013196EB30F10508F066C03F
:102EE000EC5CFF4F0C944B2D62E778E083EB95E0B0
:102EF0000E94552984E793E00E948B0D6AE578E0F3
:102F000083EB95E00E94552965E378E083EB95E03B
:102F10000E9455296BE078E083EB95E00E945529EB
:102F20006AEE77E083EB95E00E9455296DEB77E040
:102F300083EB95E00E94552967E977E083EB95E004
:102F40000E94552963E777E083EB95E00E945529BD
:102F50006CE477E083EB95E00E94552983EB95E0E4
:102F60000E9441290E94C60D21C06FE277E01AC07D
:102F70006AE077E017C065EF76E014C066ED76E0B2
:102F800011C062E976E00EC06DE776E00BC068E63E
:102F900076E083EB95E00E94552962E276E002C07C
:102FA0006CE076E083EB95E00E9455296AE070E0E2
:102FB00080E090E00E949E2783EB95E00E947B2AB0
:102FC000892B29F083EB95E00E94A82AF5CF08957C
:102FD000ACE1B0E0EEEEF7E10C941E2D90911705F8
:102FE0009F3F09F023C1482F50E0FA013A97EF368E
:102FF000F10508F00FC1E15CFF4F0C944B2D63EE1F
:1030000071E0A0C06FEE71E083EB95E00E9467294C
:1030100085E789838BE1EFE6F5E0DE01129601900A
:103020000D928A95E1F76CE1CE0101960E94360D72
:103030000E94B40C83E08093A50568EC70E080E00A
:1030400090E00E949E278091A505843009F0E2C09F
:103050008FE70E94D20A0E94E50A8983853509F02C
:10306000D9C06DEE74E083EB95E00E9455296FECBA
:1030700074E083EB95E00E94552961EB74E096C003
:1030800067E072E083EB95E00E94672989E6898317
:1030900061E0CE0101960E94360D0E94B40C83E0DF
:1030A0008093A50568EC70E080E090E00E949E2788
:1030B0008091A505843009F0ADC08FE70E94D20A47
:1030C0000E94E50A89838E010E5F1F4F7E014DE14C
:1030D000E40EF11C0E94E50AF80181938F01EE15C0
:1030E000FF05C1F78BE1FE013296AFE6B5E0019036
:1030F0000D928A95E1F78981893409F08BC063E9E3
:1031000074E083EB95E00E94552965E774E083EB5A
:1031100095E00E94552967E574E048C061E272E0DD
:1031200083EB95E00E9467298EEF8093170572C0AC
:1031300080528750805390911A05981708F066C006
:1031400060E372E083EB95E00E94672963C084E14D
:103150008093170560E274E029C085E1809317052C
:1031600069EE73E023C086E18093170562EB73E09C
:103170001DC087E18093170568E673E017C088E1FA
:103180008093170567E573E011C089E18093170507
:1031900063E473E00BC08AE1809317056EE273E08D
:1031A00005C08BE18093170566E073E083EB95E043
:1031B0000E9455292FC06CEE72E083EB95E00E94CF
:1031C000552980917D0591E01DC066ED72E083EB8D
:1031D00095E00E94552980917D0592E013C061EC35
:1031E00072E083EB95E00E94552980917D0594E083
:1031F00009C066EA72E083EB95E00E945529809150
:103200007D0598E0892780937D058FEF80931705D2
:103210000E94671083EB95E00E947B2A892B09F4BA
:103220005BC183EB95E00E94A82AF4CF0E9466114F
:10323000882309F451C18091B104811104C08FEF3A
:103240008093170541C140E050E060E070E082EB00
:1032500094E00E94C22D40911705042F112707FD0D
:103260001095212F312FF8013197EB31F10508F03E
:103270001BC1E255FF4F0C944B2D552747FD509530
:1032800020911A0530E0241735070CF40DC18B018D
:103290009C01015011092109310900321105210554
:1032A000310558F0C0901B05EDE1F5E0F12CD12C73
:1032B000A8E2EA2E415051090FC0FA01E159FA4F34
:1032C00061506083D9C0DF0111972C9130E0241741
:1032D000350729F0F3943296FC10F5CFCBC00E2DB4
:1032E00010E020E030E0061717072807390741F4FF
:1032F0002081DA01A159BA4F11962C93DD24D39481
:10330000E394E8CF6F3F71058105910511F008F056
:10331000CBC060938705B0C06F3F710581059105F3
:1033200011F008F0C1C060938805A6C06F3F710519
:103330008105910511F008F0B7C0609389059CC024
:103340002091B20420622037E9F440E050E060E0D0
:1033500070E083EB94E00E94C22D9B01AC01DC0184
:10336000CB010197A109B1090897A105B10508F0A2
:10337000AEC0A4EDB0E30E949C2C6A5E7C4A8A46F3
:10338000954E24C02636E9F440E050E060E070E05D
:1033900083EB94E00E94C22D9B01AC01DC01CB01C8
:1033A0000197A109B1090797A105B10508F08FC0E0
:1033B000A8EAB1E60E949C2C645E7C438E46944E43
:1033C00005C0611571058105910579F08B019C019E
:1033D0000054114E2D4938410138F0EF1F07FAEF24
:1033E0002F07F2E03F0708F05FC060937F057093FE
:1033F000800580938105909382053EC06F3F7105E3
:103400008105910511F008F04FC06093830534C029
:103410008B019C0101501109210931090F3F110550
:103420002105310508F040C06093840525C08B015B
:103430009C01045C1940210931090D344DE1140748
:103440002105310528F4709386056093850514C025
:10345000611571058105910521F48FEF80937E053B
:103460000BC06134710581059105F0F461506093E2
:103470007E0502C0DD20C1F08091B00481111AC028
:1034800080914F0590915005A0915105B091520542
:103490000196A11DB11D80934F0590935005A093F7
:1034A0005105B093520506C062E472E083EB95E0EB
:1034B0000E9467290E945C118FEF809317056AE0D4
:1034C00083EB95E00E9479290E94671005C061E0B6
:1034D00070E080E090E07ACF6C96E8E00C943A2DB2
:1034E0006AE572E083EB95E00E94552962E472E0A0
:1034F00083EB95E00E94552983EB95E00E947B2A9F
:10350000892B31F083EB95E00E94A82A0E94E817EE
:103510000E94C016823029F0833051F46DE072E0D1
:1035200002C064E272E083EB95E00E9455290895A1
:103530008FEF809317051092B0040E94671080915E
:1035400017058E3F69F083EB95E00E947B2A892B5B
:10355000B1F383EB95E00E94A82A0E94E817EFCF11
:1035600008950F931F93109117051F3F09F0D1C0C5
:10357000893409F457C000F5883309F468C058F459
:10358000803309F476C008F060C08B3109F440C084
:103590008132B1F1B8C0813409F486C030F4893386
:1035A00009F465C0803461F1AEC0823409F48DC085
:1035B000863409F447C0A7C0823609F486C078F47F
:1035C000883531F128F48235C1F18335E1F09BC0B3
:1035D0008A3509F493C0813609F466C094C08237F5
:1035E00061F128F4863671F18936E1F08CC08837B4
:1035F00079F08A3709F482C0833709F084C003C0A8
:1036000063EE71E015C00E94060960E672E004C036
:103610000E940F096AE772E083EB95E00E94672938
:103620008EEF6FC00E94DE070E944D0869E972E0CC
:1036300083EB95E00E94672966C00E946D0862EBEB
:1036400072E0F6CF0E9411115EC080535AC06AEF3B
:1036500071E083EB95E00E94552990916E0588E01A
:10366000890F8871977E892B80936E051AC089E037
:1036700048C067EE71E083EB95E00E945529809188
:103680008F0590919005A0919105B091920520E150
:10369000822780938F0590939005A0939105B09316
:1036A0009205109317052FC061ED71E083EB95E053
:1036B0000E94552980918F0590919005A0919105C8
:1036C000B091920540E4842710C060EC71E083EB78
:1036D00095E00E94552980918F0590919005A091C9
:1036E0009105B091920520E2822780938F059093F7
:1036F0009005A0939105B093920502C00E94701AA4
:103700008FEF80931705809117058E3F09F0D4C085
:10371000DDC00E946611882309F4D8C08091B104ED
:10372000811104C08FEF80931705C6C040E050E0C0
:1037300060E070E082EB94E00E94C22D00911705DA
:10374000112707FD1095212F312FF8013197E9300E
:10375000F10508F0B4C0E753FF4F0C944B2D8B01DB
:103760009C010154114E2D4938410F37104F2A4FFB
:10377000324008F0A4C060934B0570934C058093D1
:103780004D0590934E0577C060934F05709350059B
:10379000809351059093520581E08093B0046BC0F3
:1037A000683071058105910508F089C06093530563
:1037B00062C08B019C0101501109210931090A30B5
:1037C00011052105310508F07AC06093540553C0F6
:1037D00061EB71E082EB94E00E94FC2E10E0009718
:1037E00099F00E94D62E009779F0183130F4E12F2D
:1037F000F0E0EA5BFA4F87871F5F61EB71E080E0E2
:1038000090E00E94FC2EEBCF1831A8F5E12FF0E0FC
:10381000EA5BFA4F17861F5FF7CF653071058105A8
:10382000910508F04CC060936D0525C08B019C018B
:103830000150110921093109063011052105310511
:10384000F0F520916E05287F262B20936E0513C07E
:103850008B019C0101501109210931090115124CFC
:103860002140310560F560934705709348058093CA
:10387000490590934A058091B004811113C080914D
:103880004F0590915005A0915105B09152050196B8
:10389000A11DB11D80934F0590935005A093510534
:1038A000B09352050E945C118FEF809317056AE078
:1038B00083EB95E00E9479290E94631707C062E4B8
:1038C00072E083EB95E00E946729ECCF1F910F9186
:1038D00008958FEF809317051092B0040E9463172C
:1038E000809117058E3F69F083EB95E00E947B2A5B
:1038F000892BB1F383EB95E00E94A82A0E94B11AAC
:10390000EFCF6AE070E080E090E00E949E2783EBBA
:1039100095E00E947B2A892B29F083EB95E00E9499
:10392000A82AF5CF0895CF93C82F682F83EB95E091
:103930000E94D52A90913C059C2790933C05CF91FD
:103940000895A1E0B0E0E7EAFCE10C94242D99830E
:103950000E94931C9981892F0E94931C2196E2E07A
:103960000C94402D1F93CF93DF93182FEB011092EF
:103970003C0565EB70E083EB95E00E94590662E63A
:1039800070E083EB95E00E945906812F0E94931C02
:10399000CE010E94A11CDF91CF911F9108956091EB
:1039A0003C0583EB95E00E94D52A0895A1E2B0E0A2
:1039B000ECEDFCE10C94202D7B018A018B3009F4A5
:1039C0002DC108F03FC0853009F49BC010F582304E
:1039D00009F47EC058F4813009F02FC269E270E02A
:1039E00081E00E94B21C06E415E068C0833009F44F
:1039F00080C0843009F021C261E070E084E00E9460
:103A0000B21C81E00E94931C0E94CF1C0E94F31400
:103A10001EC2883009F49BC070F4863009F48DC052
:103A2000873009F00AC261E070E087E00E94B21CB2
:103A300080911A0508C2893009F491C08A3009F4CE
:103A4000C3C0FBC1893609F468C178F4863609F42D
:103A500019C120F4853609F401C1EFC1873609F494
:103A600025C1883609F42AC1E8C18C3609F49EC103
:103A700090F48A3609F45BC18B3609F0DEC161E04F
:103A800070E08BE60E94B21CF80180810E9435082C
:103A90000E940F09BDC18D3609F4BCC1873C09F0F5
:103AA000CCC161E070E087EC0E94B21C81E00E9412
:103AB000931C0E94CF1C10923D05C9C1F801819151
:103AC0008F010E94931CF5E00F361F07B9F7BDC1A7
:103AD0006BE170E082E00E94B21C0FE615E0F80195
:103AE00081918F010E94931CF5E00A381F07B9F7F6
:103AF000ACC161E070E083E00E94B21C0E94C0167D
:103B0000A2C160911B0570E0660F771F85E00E94DF
:103B1000B21C0CE115E080911B0590E0880F991F05
:103B200098012C5135402817390708F08EC1F8014B
:103B300081918F010E94931CEECF62E070E086E0DD
:103B40000E94B21C84E793E00E94A11C7EC161E048
:103B500070E088E00E94B21C8091A30574C186E6E3
:103B6000898361E0CE0101960E94360D0E94B40C5B
:103B700083E08093A50568EC70E080E090E00E940F
:103B80009E278091A5058430D9F48FE70E94D20A40
:103B90000E94E50A8983863469F460E270E089E076
:103BA0000E94B21C10E20E94E50A0E94931C115070
:103BB000D1F74BC161E070E089E00E94B21C28C1DE
:103BC00061E070E089E03CC169E170E08AE00E9458
:103BD000B21C10928A052091A40580918F059091C6
:103BE0009005A0919105B0919205222311F0806873
:103BF00001C08F7780938F0590939005A0939105D6
:103C0000B09392050AE815E0F80181918F010E94B6
:103C1000931CF5E0033A1F07B9F717C161E270E0A2
:103C20008BE00E94B21C80917C048F3F39F0809120
:103C30007C0491E0980F90937C0402C080917C04F6
:103C40000E94931C10E0812F0E94D4140E94640AE9
:103C50000E94A11C1F5F1031B1F7F7C061E070E056
:103C600085E60E94B21C89E2E816F10409F0EAC078
:103C7000D801E6E4F5E08D91819385E0EF36F80711
:103C8000D1F7C6C061E070E086E60E94B21CEBE1AD
:103C9000EE16F10409F0D6C0D801EFE6F5E08D91FB
:103CA000819385E0EA38F807D1F7B2C061E070E0AF
:103CB00087E60E94B21C0E940609AAC061E070E07B
:103CC00088E60E94B21C85E789838BE1EFE6F5E088
:103CD000DE01129601900D928A95E1F76CE1CE011A
:103CE00001960E94360D0E94B40C83E08093A505D6
:103CF00060E273E080E090E00E949E278091A5053D
:103D0000843009F09FC08FE70E94D20A0E94E50A22
:103D10008983853509F096C07BC061E070E089E653
:103D20000E94B21C0E94DE070E944D0871C061E033
:103D300070E08AE60E94B21C89E6898361E0CE01C8
:103D400001960E94360D0E94B40C83E08093A50575
:103D500060E273E080E090E00E949E278091A505DC
:103D6000843009F06FC08FE70E94D20A0E94E50AF2
:103D700089838E010E5F1F4F7E01EDE1EE0EF11C77
:103D80000E94E50AF80181938F01EE15FF05C1F746
:103D90008BE1FE013296AFE6B5E001900D928A9577
:103DA000E1F78981893409F04DC032C061E070E0EB
:103DB0008CE60E94B21CF0E2EF16F10461F487E693
:103DC000898380E2F801DE01129601900D928A95B6
:103DD000E1F761E203C087E4898361E0CE010196E7
:103DE0000E94360D0E94B40C83E08093A5056CE41C
:103DF00074E080E090E00E949E278091A5058430C9
:103E000009F58FE70E94D20A0E94E50A8734D1F4AF
:103E100081E019C061E070E08DE60E94B21C89E18A
:103E2000E816F10479F4D801EAE8F5E08D91819380
:103E300085E0E33AF807D1F7EBCF61E070E08AEC78
:103E40000E94B21C80E00E94931C0E94CF1CA1968D
:103E5000E6E00C943C2DA0E0B0E0E1E3FFE10C943F
:103E60001E2DCCE9D3E014E606E035E0F32E44E065
:103E7000E42E53E0D52E62E0C62E83EB95E00E943F
:103E80007B2A892B09F49BC083EB95E00E94A82A2A
:103E9000282F809307044091060450E047305105D5
:103EA00060F7FA01EE52FF4F0C944B2D853B29F73A
:103EB00081E080930604E1CF823609F07DC0C09294
:103EC0000604DBCF8093050480930404D09206049B
:103ED000D4CF9C01332730930304209302049091A4
:103EE0000404982790930404E0920604C6CF382F68
:103EF00022274091020450910304242B352B309348
:103F000003042093020490910404982790930404DE
:103F1000F09206042536310508F4AFCF61E070E079
:103F20008CEC0E94B21C81E00E94931C0E94CF1C6A
:103F300043C02091000430910104F901E456FC4F84
:103F4000808390910404982790930404C9010196FA
:103F500090930104809300042091020430910304A3
:103F60008217930708F489CF0093060486CF8091C7
:103F7000040482130BC060910004709101044CE9A9
:103F800053E0809105040E94D61C0DC062E070E0F1
:103F90008BEC0E94B21C809105040E94931C8091BE
:103FA0003C050E94931CFE01812F11928A95E9F72E
:103FB0001092010410920004109206045ECFCDB757
:103FC000DEB7E8E00C943A2D81E080933D058091C6
:103FD0003D05882349F083EB95E00E947B2A892BDD
:103FE000B1F30E942B1FF3CF0895AAE2B0E0EBEFEC
:103FF000FFE10C941C2D0E946F276B017C0181E076
:104000000E94D90B83EB95E00E947B2A892B29F033
:1040100083EB95E00E94A82AF5CF5E98409811E0C6
:1040200072E6B72EE9E2AE2E03E00E946F276C190C
:104030007D098E099F09693C710581059105E0F1B3
:104040001123D1F10E946F276B017C015D9A419A87
:1040500080ED97E00E947806B982E6E4F5E0DE01A3
:1040600012968A2D01900D928A95E1F76AE2CE01AF
:1040700001960E94360D5D98419880E090E00E9484
:1040800078060093A5050E94B40C62E370E080E01E
:1040900090E00E949E278091A505843061F40093F2
:1040A000A5058FE70E94D20A0E94E50A11E082343A
:1040B00019F410E001C011E082E10E949428892BDC
:1040C000A1F411E012C05E9A409A5D9A419A83EB86
:1040D00095E00E94A82A8D309105B9F06CF40A97FA
:1040E000A1F05E9840985D98419883EB95E00E941E
:1040F0007B2A892B41F799CF8332910579F082345D
:10410000910579F70E94E41FECCF62EB71E083EB3D
:1041100095E00E9455290E94691CE3CF0E94F31488
:10412000E0CF8F929F92AF92BF92CF92DF92EF92A9
:10413000FF921F93CF93DF9382E10E949428892BF3
:1041400009F078C068EC70E080E090E00E949E2763
:1041500080E090E00E9478060E946F274B015C018E
:104160006B017C0180ECC80E82E1D81EE11CF11CC1
:104170000E946F276C157D058E059F0530F482E146
:104180000E949428892BA1F353C082E10E949428B5
:10419000892B09F04DC080ED97E00E9478060E94BF
:1041A0006F276B017C01D0E0C1E088E4880E86E2D5
:1041B000981EA11CB11C11E082E10E949428892B59
:1041C00021F58C149D04AE04BF0430F480ED97E01B
:1041D0000E947806D1E0F0CF0E946F276C197D090C
:1041E0008E099F09693C71058105910528F30E949C
:1041F0006F276B017C01C12719F080ED97E002C0A9
:1042000080E090E00E947806D7CF80E090E00E94A6
:104210007806DD2349F08091A3058F5F83700E94AB
:1042200035080E940F0906C00E946D080E94060909
:104230000E94F51FDF91CF911F91FF90EF90DF90CB
:10424000CF90BF90AF909F908F900895CF92DF92C4
:10425000EF92FF9280E00E94DF060E94B60661E0C6
:1042600086E00E94282861E085E00E94282861E01D
:104270008EE00E94282861E08FE00E94282860E0FC
:1042800082E10E94282860E088E00E94282861E0FE
:1042900088E00E9461280E94610640E052EC61E0E3
:1042A00070E083EB95E00E94C32B0E9428080E94D7
:1042B0000F090E94B7128FEF80937C040E94CB06F7
:1042C00078940E946F276B017C0180917C048F3F62
:1042D00059F40E946F276C197D098E099F09603D72
:1042E00077408105910588F380ED97E00E9478067C
:1042F00061E082E10E9461285E9A409A83EB95E03A
:104300000E947B2A892B29F083EB95E00E94A82A42
:10431000F5CF6FEC72E083EB95E00E94362984E7DD
:1043200093E00E948B0D66EE72E083EB95E00E94B5
:1043300036294AE050E065E070E083EB95E00E94AA
:10434000062A62E370E080E090E00E949E2783EB03
:1043500095E00E947B2A04970CF183EB95E00E9484
:10436000A82A82349105D1F483EB95E00E94A82A13
:104370008E34910599F483EB95E00E94A82A843449
:10438000910561F483EB95E00E94A82A819731F4AE
:1043900080E090E00E9478060E94F51F409147055A
:1043A000509148056091490570914A05DB01CA01A9
:1043B0000197A109B1090497A105B10568F44093DB
:1043C0007B04433029F440EA56E861E070E004C021
:1043D00040E052EC61E070E083EB95E00E94C32B7B
:1043E0000E9491205E98409880E090E00E947806BC
:1043F0000E94B7121092970480918F0583FF11C01D
:1044000080915B05882351F080916205882331F00B
:1044100080916905882311F087E001C085E08093D1
:10442000970480E00E94D90B809198040E940D0BA4
:104430000E94B40C109211041092100410920F04F8
:10444000F12C8091A3058F15B0F062E370E080E05D
:1044500090E00E949E2780ED97E00E94780662E33C
:1044600070E080E090E00E949E2780E090E00E9453
:104470007806F394E6CF80916E0584FF08C0982FEC
:10448000987181E0983109F080E00E94D4118FE0AA
:104490000E94DF06FF90EF90DF90CF900895EF929B
:1044A000FF920F931F93CF93DF938C016EE770E021
:1044B00083EB95E00E945906E801F12CF0E2EF2E23
:1044C0008E0188818D57823048F46DE770E083EB70
:1044D00095E00E94590688818E2588832196F801EF
:1044E000608183EB95E00E94D52AF394F9E0FF12F6
:1044F000E7CF6EE770E083EB95E00E945906CDB7F9
:10450000DEB7E6E00C943C2DA9E0B0E0EAE8F2E288
:104510000C94242D9091990491110EC09EEF9983D3
:104520008A836B8350E0559547954C832D8319867C
:1045300018861F821E822EC040919E04842F90E018
:10454000B4E095958795BA95E1F7242F2F7030E068
:104550008217930719F18DEF89831B82FE01349630
:1045600050E0842F90E0A4E095958795AA95E1F717
:10457000242F2F7030E08217930749F0DC01A156F9
:10458000BB4F8C918193405F5F5F563051F74093F2
:104590009E045A83CE0101960E944F228091990475
:1045A00090E0019666E070E00E94BF2C8093990431
:1045B0002996E2E00C94402DA0E0B0E0E2EEF2E2B9
:1045C0000C941D2D6C016EE770E083EB95E00E946A
:1045D00059068601E12CF12CC0E0D0E030E2B32E88
:1045E000F801608183E8860F823078F46DE770E02F
:1045F00083EB95E00E945906F80160816B2570E01D
:1046000083EB95E00E94590604C083EB95E00E947D
:10461000D52AE114F10459F0F80180819E01280F98
:10462000311DC901C92FDD27C80FD91FDD273FEF75
:10463000E31AF30A89E0E816F10459F028E0E216DB
:10464000F10421F48C2F8095F60180870F5F1F4FB6
:10465000C7CFCDB7DEB7E9E00C94392DA9E0B0E0C3
:10466000E4E3F3E20C94242DE82F362F8091990493
:1046700090E0019664E270E00E94BF2C8093990460
:1046800058E9598350E15A83813089F048F08230EB
:10469000B9F08330D9F48B8381EF8C833D8319C0CB
:1046A00085E08B8381EF8C832F5F2D8312C08B83FA
:1046B00081EF8C8384E6489FA00111245D8309C0AB
:1046C00084E08B8381EF8C83ED8303C00E94111201
:1046D00004C0CE0101960E94DC222996E2E00C94EF
:1046E000402DA2E0B0E0E7E7F3E20C94192D182F7B
:1046F000762E2A8349830E947B276B017C0180915F
:10470000AF0480909A0490909B04A0909C04B09079
:104710009D042A8149818823C1F0D701C6018819E7
:104720009909AA09BB094C015D0191EE89169EE227
:104730009906A104B10420F1241708F4422F202F78
:10474000672D812F0E942E2313C0D701C60188191F
:104750009909AA09BB094C015D0191E3891695E706
:104760009906A104B10460F0672D812F0E94842274
:10477000C0929A04D0929B04E0929C04F0929D0413
:104780002296EDE00C94352DA2E2B0E0EAECF3E2E3
:104790000C941A2D8CE00E94F40A81110FC06EEE69
:1047A00072E083EB95E00E9467295E9A409A80E070
:1047B0000E94D90B0E94B40C5E98409883EB95E060
:1047C0000E947B2A892B01F183EB95E00E94A82AA5
:1047D00090917B04992319F00E94DC12EFCF409155
:1047E000100450E09A012F5F3F4F2F7133276091E3
:1047F000110470E02617370709F3FA01E55EFB4F55
:10480000808320931004DACF8091A505843009F0CD
:1048100086C00E947B27611571058105910549F0CD
:104820006093890470938A0480938B0490938C0422
:104830000CC081E090E0A0E0B0E080938904909308
:104840008A04A0938B04B0938C0480917F04909190
:10485000800481609093800480937F0483E0809340
:10486000A5058FE70E94D20A0BE314E00E94E50A37
:10487000F80181938F01F4E004341F07B9F7209108
:10488000440480913B04982F922796FF3BC090E40C
:10489000922790934404982F98739833F1F410E082
:1048A000212F30E080913B04877090E082179307BE
:1048B0004CF11F5F20916E05812F90E0FC01E55CBB
:1048C000FB4F24FF04C080810E94F311E9CF608177
:1048D00083EB95E00E94D52AE3CF8F7399F4809102
:1048E0003C048093880480913D04809386048091E9
:1048F0003E04809385048091410490E090937E046F
:1049000080937D0480910F04813019F482E08093BC
:104910000F0480910F04833011F410920F040E9451
:104920007B276B017C018091810490918204A0918E
:104930008304B09184040097A105B105C9F0A701D3
:104940009601281B390B4A0B5B0BDA01C901883B26
:104950009B40A105B10560F00E94230B8093870462
:1049600010928104109282041092830410928404A5
:1049700080918D0490918E04A0918F04B091900449
:1049800046015701881A990AAA0ABB0A86E495E0EB
:104990000E944F0986169706A806B90608F4A5C016
:1049A000C0928D04D0928E04E0928F04F092900415
:1049B0000E94570680917C048830A0F080918F057A
:1049C00090919005A0919105B09192056CE1B695FA
:1049D000A795979587956A95D1F7892B8A2B8B2B6D
:1049E00009F0ABC180917C048F5F80937C0480913F
:1049F000890490918A04A0918B04B0918C04009753
:104A0000A105B105F1F0C81AD90AEA0AFB0A86E441
:104A100095E00E944F096C157D058E059F0508F0F5
:104A200004C180918F0584FD04C080ED97E00E9451
:104A300078061092890410928A0410928B041092C6
:104A40008C0490914404907C909344045091100401
:104A50008091110420910F04581709F403C12230EA
:104A600009F000C1905890934404E0916E05E770FE
:104A7000F0E0E45BFC4F6081693008F0DBC061501E
:104A800040E04613D9C08093110487E3840F9091CE
:104A90004404892B809344044093120483E0809360
:104AA0000F045D9A419A90919704911130C18091C1
:104AB00098040E940D0BE0916E05E770F0E0E45B56
:104AC000FC4F608184E494E00E94EF0CE091980434
:104AD000EF5FE0939804E83109F42CC1F0E0EA5B61
:104AE000FA4F8785882309F425C10E945E0D813025
:104AF00069F580916E05887149F180917F049091EC
:104B00008004880F991F9093800480937F0483E032
:104B10008093A5050E94B40C0E947B2760938104BA
:104B2000709382048093830490938404672B682B92
:104B3000692B61F481E090E0A0E0B0E08093810413
:104B400090938204A0938304B093840480916E05B3
:104B500084FF1FC080917F04909180048E7F0E940B
:104B6000850A182F60917D04809188040E94D212DA
:104B7000482F612F8091870449A30E94D21200918F
:104B8000A305282F49A160918504809186040E9485
:104B900071235D984198809195048130C1F018F09F
:104BA0008230B1F1D4C082E10E949428892B09F0AF
:104BB000CEC081E0809395040E946F27609391049A
:104BC000709392048093930490939404C0C082E104
:104BD0000E949428892B31F50E946F27C090910480
:104BE000D0909204E0909304F09094046C197D09A5
:104BF0008E099F09693E73408105910508F4A7C09D
:104C000082E08093950480ED97E00E9478069FC033
:104C100082E10E949428892B09F499C080E090E0F9
:104C20000E9478061092950492C080E090E00E9465
:104C3000780607CF68E024CF851709F424CF4F5FAB
:104C4000242F30E090E0F901EC5BFB4FDC01A55E26
:104C5000BB4F7C917083F901EE5EFB4F7083019630
:104C60008F710FCF2430B1F42091120483E194E0CE
:104C7000A5E4B4E0FC013E2F381B321718F4319143
:104C80003D93F9CF87E3820F90914404892B809361
:104C9000440404CF80919504823071F49160909324
:104CA00044045E9A409A53E9E52E55E0F52E8E01B4
:104CB0000F5F1F4FB80111C05E98409880910F049C
:104CC000811103C081E080930F0480910F04833031
:104CD00051F784E080930F04E6CFF70181917F01C3
:104CE00069A37AA30E94D414F801819391938F0150
:104CF00069A17AA1F3EAEF16F5E0FF0671F780915A
:104D00006E0545E454E087700E94D409CACE8091B4
:104D10005305882309F4CBCE2091960431E0320F5D
:104D200030939604291303C01092960481500E9478
:104D3000D40BBDCE10929804D8CE80917C048830DC
:104D400011F45E9A409A89E080937C04CECEA296BC
:104D5000ECE00C94362D8230E8F4E82FF0E0EE0F12
:104D6000FF1FEA55FA4F71836083813041F08091D3
:104D700069008C7F842B80936900E89A0895809164
:104D80006900440F551F440F551F837F842B809368
:104D90006900E99A08951F920F920FB60F9211249D
:104DA0002F933F934F935F936F937F938F939F9333
:104DB000AF93BF93EF93FF938091A6059091A705C2
:104DC000892B29F0E091A605F091A7050995FF919F
:104DD000EF91BF91AF919F918F917F916F915F9173
:104DE0004F913F912F910F900FBE0F901F901895EC
:104DF0001F920F920FB60F9211242F933F934F9350
:104E00005F936F937F938F939F93AF93BF93EF9332
:104E1000FF938091A8059091A905892B29F0E09135
:104E2000A805F091A9050995FF91EF91BF91AF9168
:104E30009F918F917F916F915F914F913F912F91B2
:104E40000F900FBE0F901F9018951F920F920FB6E4
:104E50000F9211242F933F938F939F93AF93BF9300
:104E60008091AB059091AC05A091AD05B091AE05D8
:104E70003091AA0523E0230F2D3720F40196A11DC0
:104E8000B11D05C026E8230F0296A11DB11D209378
:104E9000AA058093AB059093AC05A093AD05B093A4
:104EA000AE058091AF059091B005A091B105B0918C
:104EB000B2050196A11DB11D8093AF059093B00579
:104EC000A093B105B093B205BF91AF919F918F911F
:104ED0003F912F910F900FBE0F901F9018952FB7F5
:104EE000F8946091AB057091AC058091AD059091FF
:104EF000AE052FBF08953FB7F8948091AF0590910C
:104F0000B005A091B105B091B20526B5A89B05C02A
:104F10002F3F19F00196A11DB11D3FBF6627782FC5
:104F2000892F9A2F620F711D811D911D42E0660F1E
:104F3000771F881F991F4A95D1F70895CF92DF9266
:104F4000EF92FF92CF93DF936B017C010E947B274E
:104F5000EB01C114D104E104F10479F00E947B2734
:104F60006C1B7D0B683E7340A0F381E0C81AD1082A
:104F7000E108F108C851DC4FECCFDF91CF91FF90F1
:104F8000EF90DF90CF900895789484B5826084BDCF
:104F900084B5816084BD85B5826085BD85B581603D
:104FA00085BDEEE6F0E0808181608083E1E8F0E09D
:104FB0001082808182608083808181608083E0E8CC
:104FC000F0E0808181608083E1EBF0E080818460AB
:104FD0008083E0EBF0E0808181608083EAE7F0E0AD
:104FE0008081846080838081826080838081816011
:104FF00080838081806880831092C100089583300F
:1050000081F028F4813099F08230A1F00895863043
:10501000A9F08730B9F08430D1F4809180008F7D81
:1050200003C0809180008F7780938000089584B5BD
:105030008F7702C084B58F7D84BD08958091B000C4
:105040008F7703C08091B0008F7D8093B00008956A
:10505000CF93DF9390E0FC01ED50F44F2491FC01DD
:10506000E95FF34F8491882349F190E0880F991FFD
:10507000FC01E15DF34FA591B4918B5D934FFC0171
:10508000C591D4919FB7611108C0F8948C91209577
:1050900082238C93888182230AC0623051F4F89471
:1050A0008C91322F309583238C938881822B888337
:1050B00004C0F8948C91822B8C939FBFDF91CF9189
:1050C0000895A1E0B0E0E7E6F8E20C94222D282F45
:1050D00030E0F901E152F44F8491F901ED50F44FC1
:1050E0001491F901E95FF34F04910023C9F088237B
:1050F00021F069830E94FF276981E02FF0E0EE0F25
:10510000FF1FEB5DF34FA591B4919FB7F8948C917D
:10511000611103C01095812301C0812B8C939FBF27
:105120002196E4E00C943E2DCF93DF93282F30E0BE
:10513000F901E152F44F8491F901ED50F44FD4910B
:10514000F901E95FF34FC491CC2391F081110E94E2
:10515000FF27EC2FF0E0EE0FFF1FE55EF34FA59168
:10516000B4912C912D2381E090E021F480E002C0E5
:1051700080E090E0DF91CF9108958E3008F08E505E
:10518000877020919D0190E4299F90011124822B2A
:1051900080937C0080917A00806480937A00809173
:1051A0007A0086FDFCCF809178002091790090E014
:1051B000922B0895A0E0B0E0E0EEF8E20C941E2DF2
:1051C0006C017A01EB01E60EF71E00E010E0CE154F
:1051D000DF0561F06991D601ED91FC910190F081BC
:1051E000E02DC6010995080F191FF1CFC801CDB7F1
:1051F000DEB7E8E00C943A2D6115710589F0DB010A
:105200000D900020E9F7AD0141505109461B570BA5
:10521000DC01ED91FC910280F381E02D0995089568
:1052200080E090E00895EF92FF920F931F93CF9349
:10523000DF938C01FB01C0E0D0E064917F018FEF30
:10524000E81AF80A662361F0D801ED91FC9101900B
:10525000F081E02DC8010995C80FD91FF701EDCFE6
:10526000CE01CDB7DEB7E6E00C943C2D0E94FC28C1
:105270000895DC01ED91FC910190F081E02D0995FC
:1052800008950F931F93CF93DF93EC016DE00E947D
:1052900039298C016AE0CE010E943929800F911FC3
:1052A000DF91CF911F910F9108950F931F93CF938B
:1052B000DF93EC010E9413298C01CE010E94412949
:1052C000800F911FDF91CF911F910F9108950F9340
:1052D0001F93CF93DF93EC010E94FC288C01CE0139
:1052E0000E944129800F911FDF91CF911F910F9153
:1052F00008950F931F93CF93DF93EC010E943929F8
:105300008C01CE010E944129800F911FDF91CF9126
:105310001F910F910895A1E2B0E0E1E9F9E20C9448
:105320001A2D7C01C42EE52FCB01D22E19A221E02B
:105330002D1510F02AE0D22E8E010F5D1F4F8D2CFF
:10534000912CA12CB12C6C2D7E2FA50194010E94D3
:10535000D32C8C2DD29E80191124015011098A3032
:1053600010F4805D01C0895CF8018083211531054E
:105370004105510521F0C22EE32FCA01E4CFB80147
:10538000C7010E94FC28A196ECE00C94362DA0E009
:10539000B0E0EDECF9E20C941E2DEC016A017B010A
:1053A0002115310541F4E881F9810190F081E02D6A
:1053B000642F09951DC02A303105A9F477FF12C06A
:1053C0006DE20E9439298C0144275527BA014C19F6
:1053D0005D096E097F092AE0CE010E948B29800FAA
:1053E000911F06C02AE0B701A601CE010E948B29B9
:1053F000CDB7DEB7E8E00C943A2D9A01AB016627F1
:1054000057FD6095762F0E94C72908950F931F932B
:10541000CF93DF93EC019A01AB01662757FD6095AE
:10542000762F0E94C7298C01CE010E944129800F4E
:10543000911FDF91CF911F910F9108952115310593
:1054400049F4DC01ED91FC910190F081E02D642F95
:10545000099508950E948B2908959A01462F50E0DE
:1054600060E070E00E941E2A08959A01AB0160E09E
:1054700070E00E941E2A08950F931F93CF93DF932D
:10548000EC010E941E2A8C01CE010E944129800F4E
:10549000911FDF91CF911F910F9108950F931F934B
:1054A000CF93DF93EC019A01AB0160E070E00E94C2
:1054B0001E2A8C01CE010E944129800F911FDF918D
:1054C000CF911F910F9108950F931F93CF93DF9367
:1054D000EC019A01462F50E060E070E00E941E2A25
:1054E0008C01CE010E944129800F911FDF91CF9145
:1054F0001F910F910895FC0124853585F901E05C29
:10550000FF4F80819181F901EE5BFF4F2081318156
:10551000821B930B8F7399270895FC0184859585D1
:10552000FC01E05CFF4F40815181FC01EE5BFF4FCD
:10553000208131814217530741F00190F081E02D25
:10554000E80FF91F808190E008958FEF9FEF089595
:10555000FC0184859585FC01E05CFF4F4081518111
:10556000FC01EE5BFF4F208131814217530779F038
:10557000A081B181A80FB91F8C91208131812F5F4B
:105580003F4F2F7333273183208390E008958FEFAF
:105590009FEF0895FC0181A1882329F0A489B58992
:1055A0008C9186FFFBCF11A20895CF93DF93FC016E
:1055B00026853785D901A05CBF4F8D919C911197AD
:1055C00001968F739927E901CE5BDF4F488159819E
:1055D00084179507D9F30D90BC91A02DA20FB31F8E
:1055E0006C93A685B785A05CBF4F11969C938E9354
:1055F000A689B7892C9181E090E0078C02C0880FC2
:10560000991F0A94E2F7282B2C9381E081A3048848
:10561000F589E02D80818064808381E090E0DF91D6
:10562000CF91089508951F920F920FB60F921124F3
:105630002F933F934F938F939F93EF93FF9380917B
:10564000C00082FD1CC04091C60080915906909117
:105650005A0601968F73992720915B0630915C065C
:105660008217930771F0E0915906F0915A06E75EB0
:10567000F94F408390935A068093590602C0809157
:10568000C600FF91EF919F918F914F913F912F9184
:105690000F900FBE0F901F90189583EB95E00E941E
:1056A0007B2A892B11F00E94122B08951F920F92D2
:1056B0000FB60F9211242F933F938F939F93EF93E5
:1056C000FF93209115063091160680911706909150
:1056D00018062817390731F48091C1008F7D809317
:1056E000C10014C0E0911706F0911806EB52FA4F72
:1056F0002081809117069091180601968F73992743
:1057000090931806809317062093C600FF91EF919F
:105710009F918F913F912F910F900FBE0F901F90EF
:105720001895A0E0B0E0E7E9FBE20C941A2DFC012B
:105730001382128288EE93E0A0E0B0E08483958328
:10574000A683B7838EE893E091838083758764870F
:1057500057874687318B208B138B028BF58AE48A1F
:10576000D78AC68AB18EA08E938E828E8F85848FC3
:105770008889858F8989868F8A89878F8B8980A37D
:10578000ECE00C94362DCF92DF92EF92FF92CF9304
:10579000DF93EC016A017B01411581EE5807610539
:1057A0007105F9F0EC89FD8981E090E008A002C064
:1057B000880F991F0A94E2F7808360E079E08DE317
:1057C00090E0A70196010E94D32C21503109410994
:1057D00051095695479537952795211580E138074A
:1057E00098F0EC89FD89108260E874E88EE190E021
:1057F000A70196010E94D32C21503109410951097A
:105800005695479537952795E889F9893083EA8930
:10581000FB89208319A2EE89FF89408181E090E015
:105820009C010C8C02C0220F331F0A94E2F7422B1A
:105830004083EE89FF8940819C010D8C02C0220FBC
:10584000331F0A94E2F7422B4083EE89FF8940819F
:105850009C010E8C02C0220F331F0A94E2F7422BE8
:105860004083EE89FF8920810F8C02C0880F991F29
:105870000A94E2F7809582238083DF91CF91FF9095
:10588000EF90DF90CF9008958F929F92AF92BF924A
:10589000CF92DF92EF92FF920F931F9381E08F934D
:1058A00085E08F9387E08F9383E08F9384E08F93DD
:1058B000E6EC8E2E912CF2ECAF2EB12CA1ECCA2E80
:1058C000D12CB0ECEB2EF12C04EC10E025EC30E008
:1058D00045ED55E069E176E083EB95E00E94912B80
:1058E0000F900F900F900F900F901F910F91FF90BE
:1058F000EF90DF90CF90BF90AF909F908F900895E2
:105900000E94C4270E942621CDE4DBE20E94C4232A
:105910002097E1F30E944D2BF9CFA29FB001B39FD6
:10592000C001A39F700D811D1124911DB29F700DA8
:10593000811D1124911D08950E948D2CA59F900D0D
:10594000B49F900DA49F800D911D11240895B7FF61
:105950000C949C2C0E949C2C821B930B0895DB01C1
:105960008F939F930E949C2CBF91AF91A29F800D1B
:10597000911DA39F900DB29F900D1124089597FB48
:10598000072E16F4009407D077FD09D00E94512D00
:1059900007FC05D03EF4909581959F4F0895709532
:1059A00061957F4F0895A1E21A2EAA1BBB1BFD0132
:1059B0000DC0AA1FBB1FEE1FFF1FA217B307E407EE
:1059C000F50720F0A21BB30BE40BF50B661F771F46
:1059D000881F991F1A9469F7609570958095909526
:1059E0009B01AC01BD01CF010895052E97FB1EF46C
:1059F00000940E940C2D57FD07D00E94D32C07FC69
:105A000003D04EF40C940C2D509540953095219573
:105A10003F4F4F4F5F4F08959095809570956195DA
:105A20007F4F8F4F9F4F08952F923F924F925F92DB
:105A30006F927F928F929F92AF92BF92CF92DF929E
:105A4000EF92FF920F931F93CF93DF93CDB7DEB703
:105A5000CA1BDB0B0FB6F894DEBF0FBECDBF099497
:105A60002A88398848885F846E847D848C849B84EE
:105A7000AA84B984C884DF80EE80FD800C811B81FC
:105A8000AA81B981CE0FD11D0FB6F894DEBF0FBE2B
:105A9000CDBFED010895EE0FFF1F0590F491E02DAD
:105AA0000994AA1BBB1B51E107C0AA1FBB1FA61765
:105AB000B70710F0A61BB70B881F991F5A95A9F7B7
:105AC00080959095BC01CD0108958F929F92AF92E1
:105AD000BF92CF92DF92EF92FF92CF93DF93EC01D0
:105AE000688179818A819B816115710581059105A4
:105AF00021F464E279ED8BE597E02DE133EF41E0AD
:105B000050E00E94F52C49015A019B01AC01A7EA23
:105B1000B1E40E949C2C6B017C01ACEEB4EFA501BA
:105B200094010E94AA2CC60ED71EE81EF91EF7FE8D
:105B300006C081E0C81AD108E10880E8F80AC882E6
:105B4000D982EA82FB82C701B6019F77DF91CF91AC
:105B5000FF90EF90DF90CF90BF90AF909F908F908D
:105B600008950E94652D089586E091E00E94652DBC
:105B70000895609306017093070180930801909344
:105B8000090108952F923F925F926F927F928F92B8
:105B90009F92AF92BF92CF92DF92EF92FF920F93BC
:105BA0001F93CF93DF938B01EA016115710521F0FB
:105BB000DB018C9311969C93209739F09E01225023
:105BC00031092332310508F0D8C07C016701BFEFED
:105BD000CB1ADB0A5601F7016080862D90E00E9407
:105BE000F42E892B11F07601F1CFFDE26F120AC07D
:105BF000570182E0A80EB11CD70111966C90772452
:105C000073940BC0BBE26B1207C05701E2E0AE0E0B
:105C1000B11CD70111966C90712CCE018F7E892B0F
:105C200089F4B0E36B1237C0F50180818F7D883530
:105C3000D1F46180F2E0AF0EB11C872D8260782E26
:105C4000C0E1D0E0CA30D10551F1C031D10521F019
:105C5000C830D10599F409C0CC24CA94DC2CEC2CB2
:105C6000AFE0FA2E22C0209769F7C8E0D0E0CC243C
:105C7000CA94DC2CEC2CFFE1FF2E17C06FEF7FEFF6
:105C8000CB019E01442737FD4095542F0E94D32C11
:105C900069017A010AC02097A9F6CAE0D0E0E9E9D3
:105CA000CE2EDC2CEC2CE9E1FE2EF50160E020E0AC
:105CB00030E0A9014E01AA2497FCA094BA2C1F0140
:105CC00070ED572E560CA9E0A51570F48FEB860DDC
:105CD0008A3118F499EC592E06C08FE9860D8A3165
:105CE00048F589EA582E560C852D90E08C179D07B3
:105CF0000CF56F3FD9F0C216D306E406F50698F00E
:105D0000C501B4010E94AF2C9B01AC01852D90E030
:105D1000A0E0B0E0280F391F4A1F5B1F2817390782
:105D20004A075B0710F46FEF01C061E03196D101C3
:105D30006C90C5CF0115110551F0662311F0319714
:105D400003C071FE04C03297D801ED93FC9370FE3E
:105D500007C050954095309521953F4F4F4F5F4F6D
:105D600067FF10C082E290E090935E0680935D062C
:105D70006FEF7FEF8FEF9FEF07C060E070E080E094
:105D800090E002C0B901CA01DF91CF911F910F913C
:105D9000FF90EF90DF90CF90BF90AF909F908F904B
:105DA0007F906F905F903F902F900895FC0188271F
:105DB0009927E89421912032E9F3293010F02E3010
:105DC000C8F32B3241F02D3239F4689404C00E949C
:105DD000282F820F911D219120532A30C0F31EF4E9
:105DE000909581959F4F0895911150C0803219F080
:105DF00089508550D0F708954AE953E00E94012F59
:105E00000895FA01A191B081009719F41097E1F07B
:105E1000CD01DC01CD010D90002011F4C00113C0B3
:105E2000FB012191222319F02015D9F7F3CFFB01B3
:105E30002191201519F41E92119606C02223C1F754
:105E40000D900020A1F7D001FA01A193B08308952D
:105E50007AE0979F902D879F802D910D11240895B2
:105E6000F999FECF92BD81BDF89A992780B5089522
:105E7000262FF999FECF1FBA92BD81BD20BD0FB666
:105E8000F894FA9AF99A0FBE0196089599278827EF
:065E90000895F894FFCF15
:105E960000005F06200001000000FF000200020073
:105EA60002000200020002000200020002000200DC
:105EB6000200020002000200020002802500000526
:105EC600400AA1204EA50020244EA52C2330C01246
:105ED60000001A400AA1204EA5001B1E27522C23A3
:105EE600308025000005400AA1204EA50020244E42
:105EF600A52C2330004B000006400AD0009D490027
:105F06007B289D492C233000E1000005400A45010D
:105F1600D7DC03B81E0EBF00232E48E801008A40D6
:105F26000A6001555502AD1E20000023C8015458D1
:105F36002074696D656F75742100596573004E6F25
:105F4600002C00386368004E2F41002C205B005D5A
:105F56002028002900486F70206368616E6E656CAA
:105F66002000204020007363616E6E6572206D6FA5
:105F76006465004E4F5420454E41424C4544005303
:105F8600656E64696E672073657474696E677320E5
:105F9600746F2052580A00526573657474696E678F
:105FA6002073657474696E6773206F6E2052580A89
:105FB6000041626F727465642065646974730A00D7
:105FC600696E76616C69642073656C656374696F6C
:105FD6006E000D0A496E76616C696420696E707593
:105FE60074202D20646973636172646564210700FF
:105FF60053657474696E6773207361766564207483
:106006006F20454550524F4D0A00526576657274B1
:1060160065642073657474696E67732066726F6D4C
:1060260020454550524F4D0A004C6F61646564200F
:10603600666163746F72792064656661756C7473EA
:106046000A004B657920616E64206368616E6E6537
:106056006C732072616E646F6D697A65640A004FB5
:1060660070656E4C52536E6720545820737461727B
:1060760074696E672000206F6E20485720006D6F90
:1060860064756C65206C6F636B65643F00342B34FC
:10609600003800382B340031320031322B340031D5
:1060A600360050504D00525353490053444100535B
:1060B600434C00525844005458440041494E004C49
:1060C600424545500053504B54524D005342555390
:1060D6000053554D44004C4C494E440000070B0CF0
:1060E60010111500B701FD020103030307030A039C
:1060F6000F03B701160A13223129120316031B03D5
:106106001F03230327032B032F0335033C034103FC
:1061160046035F025F025F025F0200000000D52AAD
:0A612600DA287B2AA82A8D2ACA2A4B
:00000001FF
